:1000000000308A00CE2900000A108A100A118207E7
:1000100028340C34013406340A108A100A1182077D
:10002000413468346F346A3400341C308400000872
:100030000319292801308D008C018C0B1D288D0B94
:100040001C284A308C008C0B232800000000800BF9
:100050001A2800340608C339A300220D8C008C0D29
:10006000FC308C050C083C392304860006148316EA
:100070000610000083120610831606108312003447
:10008000A008031D4528861046288614831686106E
:100090008312A10E2108A2002A20A10E2108A2008D
:1000A0002A200D308C008C0B5328003414309C0017
:1000B0001520C3308316860583128610831686109A
:1000C0008312061083160610831299011908023C48
:1000D000031C722802309C0015200330A2002A2045
:1000E000990A66280D308C008C0B74280230A2000F
:1000F0002A200D308C008C0B7B2899011908023CBA
:10010000031C8E28190804209A00A0011A08A100D7
:10011000402002309C001520990A7E28D229013007
:100120001C029E001D08023C031D982840309E07BB
:100130001E0880389F00A0011F08A1004020003445
:100140001B088C000C300C020319B3280A300C0277
:100150000319BB280D300C020319C12808300C020A
:100160000319C628CB28A0010130A100402002308D
:100170009C001520D72801309C0002309D008F2064
:10018000D72801309C009D008F20D728A001103077
:10019000A1004020D7281B081F3C031CD128073092
:1001A0009B050130A0001B08A1004020D728003487
:1001B0001E088400800104309F009F080319EE2868
:1001C000831685158312851DE72804309F0029308A
:1001D0008C008C0BE92800009F03DD288316851511
:1001E0008312851DEE28DD308C008C0BF528000075
:1001F00000001D08840083168515003083128519C0
:10020000013080009F011F08033C031C2829A630F1
:100210008C008C0B092900001E0884000310000CC0
:100220008C008000831685158312851D1C291E08ED
:10023000840008300007800020182029051121299A
:1002400005158316051101308312A0069F0A0329A4
:1002500000308D0000341B309D001A089E00D8200D
:100260008D080319362901308D0086299B08031D4E
:100270002B291A08840000080F3C03194229023078
:100280008D0086291B309D0019089E00D8208D08FE
:1002900003194D2901308D0086299B08031D532920
:1002A00003308D0086291B309D001A089E00D8203F
:1002B0008D0803195E2901308D0086299B08031DD6
:1002C000642903308D0086291B309D001C309E0060
:1002D000D8208D0803196F2901308D0086299B08CD
:1002E000031D752903308D00862919088400000834
:1002F0009D001A08840000081D070F391C0203190D
:10030000842903308D00862900308D00FA291C08CD
:100310008D011B0203188F291B088C009B298C015F
:1003200008309D009B0D8C0D1C080C0203188C00DE
:100330008D0D9D0B922900340D0819089B00643027
:100340009C0087210C0899000D083030031DAF294F
:100350001A189A159A19B5291A1A2030B1299A1122
:100360001A128D070D089B00A02019089B000A3067
:100370009C0087210C0899000D083030031DC4290A
:100380009A19C8291A1A20308D070D089B00A02041
:100390003030990719089B00A020003484011F30D9
:1003A0008305562805309C001520990119080C205A
:1003B000990A9B00A02004301902031DD62903309E
:1003C0009A002E309B00A0209A0BE1290230990060
:1003D00096309C001520990BE8298E018F01900121
:1003E0009101920193019401950116309900173003
:1003F0009A002B290D0898009808031D102A013037
:100400001602FD3E0318102A033EA82A17088E0084
:10041000900A102A17088F00910A102A950A102AAC
:1004200001309C009D008F2058309B00A0200E08BA
:10043000990011309A009C2120309B00A0201008C8
:10044000990010309A009C211208990010309A00EF
:100450009C211808990010309A009C2120309B00A4
:10046000A02020309B00A02001309C0002309D0085
:100470008F2059309B00A0200F08990011309A005E
:100480009C2120309B00A0201108990010309A0078
:100490009C211408990010309A009C21170899009B
:1004A00010309A009C2120309B00A02020309B001F
:1004B000A020831605108312051401309C0015201E
:1004C0000E08970017089703003A0319712A153090
:1004D0008C008C0B692A00009708031D702A0030DD
:1004E000622A831605108312051083168510831265
:1004F000851401309C0015200F08970017089703FA
:10050000003A03198D2A15308C008C0B852A0000C7
:100510009708031D8C2A00307E2A831685108312CB
:1005200085100E081E3C8D000F080D02970017085D
:100530009703003A0319A62A15308C008C0B9E2ACB
:1005400000009708031DA52A0030972AF5296300AB
:0E0550000A108A140A118207062A0A2A0E2AA5
:02400E00F13F80
:00000001FF
